:020000040800F2
:100000007806002029020008FF0C00087D0C00087B
:10001000FD0C00081F040008A90D000800000000E6
:10002000000000000000000000000000030D0008B8
:100030002104000800000000010D0008050D000863
:10004000430200084302000843020008430200087C
:10005000430200084302000843020008430200086C
:10006000430200084302000843020008430200085C
:10007000430200084302000843020008430200084C
:10008000430200084302000843020008430200083C
:10009000430200084302000843020008430200082C
:1000A000430200084302000843020008430200081C
:1000B000430200084302000843020008430200080C
:1000C00043020008430200084302000843020008FC
:1000D00043020008430200084302000843020008EC
:1000E00043020008430200084302000843020008DC
:1000F00043020008430200084302000843020008CC
:1001000043020008430200084302000843020008BB
:1001100043020008430200084302000843020008AB
:10012000430200084302000843020008430200089B
:10013000430200084302000843020008430200088B
:10014000430200084302000843020008430200087B
:10015000430200084302000843020008430200086B
:10016000430200084302000843020008430200085B
:100170004302000843020008430200080000000098
:10018000430200084302000800F002F800F03CF8C7
:100190000AA090E8000C82448344AAF10107DA45E2
:1001A00001D100F031F8AFF2090EBAE80F0013F0F8
:1001B000010F18BFFB1A43F001031847A00C000001
:1001C000C00C0000103A24BF78C878C1FAD8520792
:1001D00024BF30C830C144BF04680C6070470000C1
:1001E0000023002400250026103A28BF78C1FBD840
:1001F000520728BF30C148BF0B6070471FB500F0E1
:100200001FFE1FBD10B510BD00F0CFF81146FFF75F
:10021000F5FF00F0F9FD00F0EDF803B4FFF7F2FF91
:1002200003BC00F0F5F80000094880470948004782
:10023000FEE7FEE7FEE7FEE7FEE7FEE7FEE7FEE796
:10024000FEE7FEE704480549054A064B70470000F3
:10025000990D000889010008780000207806002028
:10026000780200207802002053EA020C00F0698036
:100270002DE9F04B4FF00006002B1FBFB3FA83F5BA
:1002800003FA05F424FA05F65E4012BF1643B2FAEB
:1002900082F502FA05F4C5F120051EBF22FA05FC1D
:1002A00044EA0C04203556EA044C4FEA144418BFC3
:1002B000641C4FF000084FF00009904271EB030CF2
:1002C00039D3002919BFB1FA81F701FA07F6B0FA5C
:1002D00080F700FA07F6C7F120071EBF20FA07FCD7
:1002E00046EA0C062037B6FBF4FCA7EB0507103FE7
:1002F00007F01F0BCBF120060CFA0BFB2CFA06F6CD
:1003000044BFB3460026202FA4BF5E464FF0000B2B
:100310005BEA060C08BF4FF0010B19EB0B09ABFBB6
:10032000027C48EB0608C01B06FB02CC0BFB03CC8F
:1003300071EB0C01C1E70B46024641464846BDE859
:10034000F08B13B54FF000004FF00001AFF30080C9
:10035000BDE81C4070474FF0000200B513469446BC
:100360009646203922BFA0E80C50A0E80C50B1F10D
:100370002001BFF4F7AF090728BFA0E80C5048BF21
:100380000CC05DF804EB890028BF40F8042B08BFBF
:10039000704748BF20F8022B11F0804F18BF00F8BB
:1003A000012B7047704770477047754600F02CF876
:1003B000AE4605006946534620F00700854618B052
:1003C00020B5FFF73FFFBDE820404FF000064FF09B
:1003D00000074FF000084FF0000B21F00701AC467A
:1003E000ACE8C009ACE8C009ACE8C009ACE8C00999
:1003F0008D46704710B50446AFF300802046BDE837
:100400001040FFF70ABF00000048704714000020AA
:1004100001491820ABBEFEE7260002007047FEE748
:10042000704700002DE9F84FDFF8BCA1002201253C
:1004300003264FF00F090AF1040BAAF1040E00BFC6
:100440000B6805FA02F42340A34270D10F7907F03C
:100450000307012F01D0022F16D187684FEA420807
:1004600006FA08FC27EA0C07D1F80CC00CFA08FCC5
:100470004CEA070CC0F808C04768A7430C79C4F3DE
:10048000001494403C4344600C79E443A4070AD030
:10049000C4684FEA420C06FA0CF7BC438F6807FAAF
:1004A0000CF72743C7600C7904F00304022C12D127
:1004B000D40800EB840CDCF820405707FF0E09FA43
:1004C00007F824EA0804D1F8108008FA07F848EA87
:1004D0000408CCF8208004684FEA420C06FA0CF7B6
:1004E000BC430F7907F0030707FA0CF727430760AF
:1004F0004C6814F4403F70D03C4C276847F4804768
:100500002760246822F0030704F480440094384CE8
:1005100007EB040CDCF8084897074FEA177809FA4C
:1005200008F7BC43334FB84202D1002724E054E01F
:10053000314FB84201D101271EE0304FB84201D1FE
:10054000022719E02E4FB84201D1032714E02D4FA6
:10055000B84201D104270FE02B4FB84201D1052743
:100560000AE02A4FB84201D1062705E0284FB842D9
:1005700001D1072700E0082707FA08F72743CCF83E
:100580000878DAF800405746D1F804C09C435FEA87
:10059000CC2C00D51C433C60DBF800405F46D1F812
:1005A00004C09C435FEA8C2C00D51C433C60DEF801
:1005B00000407746D1F804C09C435FEA8C3C00D5EC
:1005C0001C433C60084F083F3C68D1F804C09C4382
:1005D0005FEACC3C00D51C433C60521C102AFFF45F
:1005E0002FAFBDE8F88F0000083C014044380240BE
:1005F00000300140000002400004024000080240B8
:10060000000C02400010024000140240001802409A
:10061000001C0240426921EA02030A4043EA024107
:10062000816170470AB1816170470904FBE70000EE
:10063000014880687047000004000020024881687B
:100640000278114481607047040000200B4810B507
:10065000016841F400710160016841F4806101604A
:10066000016841F480710160032000F061F80F20FF
:1006700000F006F800F024F8002010BD003C024015
:1006800070B50D4D04464FF47A712878B1FBF0F047
:100690000A490968B1FBF0F000F0DCFA48B9102C07
:1006A00007D200222146501E00F022F800206C6084
:1006B00070BD012070BD000004000020100000206B
:1006C0000A4808B5016841F480410160006800F4FF
:1006D000804000900548001F016841F08051016092
:1006E000006800F08050009008BD000044380240CF
:1006F000F0B40E4B1B680C46C3F30223C3F107058D
:10070000042D00D90425191D072901D2002300E07A
:10071000DB1E012606FA05F1491E214099409E4044
:10072000761E16403143F0BC00F03FBB0CED00E0FC
:10073000064900F0070208684FF6FF03184040EA38
:100740000220034A10430860704700000CED00E0EF
:100750000000FA052DE9F0470E46050065D0DFF8E8
:100760001481D8F80000F7B200F00700B04207D2B9
:1007700088F80070D8F8000000F00700B04254D1AB
:1007800028683D4C810712D5400703D5206840F406
:10079000E05020602878000703D5206840F46040CE
:1007A00020602068A96820F0F000084320602878C5
:1007B000C0072DD0304968680839012812D00228B6
:1007C00013D0032811D00968890700292DDA216880
:1007D00021F0030101432160FFF72AFF814641F226
:1007E000883A0EE009688903EFE709688901ECE7B8
:1007F000FFF71EFFA0EB0901514502D90320BDE818
:10080000F0872068696800F00C00B0EB810FEFD131
:10081000D8F80010404601F00701B14207D907702F
:10082000006800F00700B04201D00120E7E7287817
:10083000400705D52068E96820F4E05008432060AF
:100840002878000706D52068296920F4604040EA2E
:10085000C100206000F018F82168084AC1F30311B4
:10086000515CC8400649086006480068FFF708FF69
:100870000020C4E7003C0240083802404A0E00084D
:100880001000002008000020154810B5006810F086
:100890000C02144813D04110042A0FD0082A0ED19C
:1008A0000F4C241F2268236802F03F025B0207D529
:1008B0002068C0F38810A0FB010106E0084610BDC7
:1008C0002168C1F38811A1FB00010023FFF7CCFCD4
:1008D0002168C1F30141491C4900B0FBF1F010BD92
:1008E000083802400024F4002DE9F84F04006ED0CF
:1008F0002078DFF84C93C007A9F104054AD009F12C
:1009000004000168C1F38101012908D00068C0F327
:10091000810002280AD1D9F80000400206D52868D3
:10092000800337D560680028E1D033E06068B0F517
:10093000803F10D0B0F5A02F286810D020F4803070
:100940002860286820F4802028606068A8B1FFF73C
:100950006FFE06460DE0286840F48030F4E740F46E
:1009600080202860F7E700BFFFF762FE801B642845
:1009700073D828688003F7D50CE0FFF759FE0646C8
:1009800005E000BFFFF754FE801B6428F0D82868FC
:100990008003F7D42078DFF8AC8280074FF0000A9C
:1009A0003ED5A748001D016811F00C0F08D0006863
:1009B000C0F3810002280BD1D9F80000400207D40F
:1009C0002868800716D5E068012800D112E033E1DD
:1009D000E068B8B10120C8F80000FFF729FE06461C
:1009E00005E000BFFFF724FE801B0228C0D828685E
:1009F0008007F7D52868216920F0F80040EAC10097
:100A000028600DE0C8F800A0FFF712FE064604E0DB
:100A1000FFF70EFE801B02281FD828688007F7D436
:100A20002078000722D5864F87486169703771B1F9
:100A300001210160FFF7FCFD064604E0FFF7F8FD29
:100A4000801B022809D838688007F7D50EE0C0F867
:100A500000A0FFF7EDFD064605E082E0FFF7E8FDA8
:100A6000801B02287DD838688007F7D4207840079B
:100A700068D5DFF8CCB100270BF13C0BDBF80000A8
:100A8000C0000BD4DBF8001041F08051CBF800100F
:100A9000DBF80000012700F0805000906B4E3068BA
:100AA000C00510D4306840F480703060FFF7C0FD9E
:100AB000009005E0FFF7BCFD0099401A022850D8CD
:100AC0003068C005F6D55E4EA0686C3601280FD0A0
:100AD0000528306810D020F001003060306820F028
:100AE00004003060A068B8B1FFF7A2FD00900FE0ED
:100AF000306840F00100F4E740F004003060F7E7B0
:100B0000FFF796FD0099411A41F28830814266D87C
:100B100030688007F4D50EE0FFF78AFD009007E00B
:100B2000FFF786FD0099411A41F28830814256D87C
:100B300030688007F4D42FB1DBF8001021F0805129
:100B4000CBF80010A069C8B33D49091D0968C1F37D
:100B5000810102294AD00228504607D0C8F8600017
:100B600000E03CE0FFF764FD04463BE04746C8F880
:100B70006000FFF75DFD064605E000BFFFF758FD8A
:100B8000801B02282BD828688001F7D4D4E90701FC
:100B90000843A16A2E4A490802EB0141626A41EA10
:100BA0008211084394F82C1040EA0161C9F8001042
:100BB00001203866FFF73CFD044606E03EE000BF3A
:100BC000FFF736FD001B022809D828688001F7D5F9
:100BD00034E000BFFFF72CFD001B022802D90320E0
:100BE000BDE8F88F28688001F4D427E00128F7D009
:100BF000D9F80000E26900F4800191421CD1226A18
:100C000000F03F01914217D147F6C071626A01407E
:100C1000B1EB821F10D1A26A4FF0FF3300F44031D4
:100C200003EB5202B1EB024F06D194F82C1000F006
:100C30007060B0EB016F01D00120D1E70020CFE759
:100C40000438024000004742800E474200700040D6
:100C50000000FFFF10B5401EB0F1807F01D30120DE
:100C600010BD4FF0E02460610F21601700F09DF887
:100C70000020A06107202061002010BDFEE70000D9
:100C800070B586B014216846FFF765FB1948016806
:100C900041F004010160016801F00401059101685F
:100CA00041F080010160016801F080010591016857
:100CB00041F00101016000680F4E00F00100059055
:100CC000012230213046FFF7ADFC1020012402251F
:100CD0008DE83100694630460395FFF7A3FB2020DD
:100CE000CDE9000469463046CDE90245FFF79AFB9D
:100CF00006B070BD3038024000080240FEE7FEE753
:100D000070477047FFF79ABC30B593B03021684602
:100D1000FFF721FB14210CA8FFF71DFB1C48002442
:100D2000016841F080510160006800F0805011902E
:100D30001848016841F4804101600068022500F410
:100D40008040119001200090000401908001CDE9C5
:100D500006500420A821CDE908010A900B906846AE
:100D6000FFF7C2FD08B172B6FEE70F20CDE90C0512
:100D70004FF48050CDE90E4002210CA81094FFF7EB
:100D8000E9FC002801D072B6FEE713B030BD0000C8
:100D900040380240007000400248016841F4700190
:100DA0000160704788ED00E0FEE70907090E0028A2
:100DB00004DB00F1E02080F80014704700F00F0021
:100DC00000F1E02080F8141D70474FF47A71484319
:100DD000AFF3008070B54FF0E02400226569094947
:100DE000A36909684843A1699942FCD002D2A3EBE8
:100DF000010302E0A5EB010633441A440B4682428C
:100E0000F1D370BD00000020FFF720FCFFF77CFF4E
:100E1000FFF736FF08495420084C4FF4FA75086074
:100E200010212046FFF7F6FB20212046FFF7F2FBBA
:100E30002846FFF7CAFFF3E7000000200004024045
:100E40004FF04070E1EE100A704700000000000013
:100E50000000010203040607080900007C0E0008D8
:100E60000000002014000000C4010008900E0008DB
:100E70001400002064060000E001000800000000EB
:100E80000100000010000000000000000024F40039
:040000050800018965
:00000001FF
